:04000000DCEF00F041
:100008004582FACF05F0FBCF06F0E9CF07F0EACF3B
:1000180008F0E1CF09F0E2CF0AF0D9CF0BF0DACF40
:100028000CF0F3CF0DF0F4CF0EF0F6CF0FF0F7CFC2
:1000380010F0F8CF11F0F5CF12F045C013F046C01C
:1000480014F047C015F048C016F083969EA289D0D8
:1000580080CF18F0070E196E1950020D250EF324E3
:10006800D96E000EF420DA6EDECF01F0DDCF02F09B
:10007800D8900136023619C003F018C004F0032ADC
:1000880002D0D8900432032EFCD7010E0416045077
:100098000112000E02121950020D250EF324D96E1A
:1000A800000EF420DA6E01C0DEFF02C0DDFF190683
:1000B8001928D8A4D1D781CF18F0070E196E195076
:1000C800020D250EF324D96E000EF420DA6EDECF71
:1000D80001F0DDCF02F0D8900136023619C003F0E6
:1000E80018C004F0032A02D0D8900432032EFCD79B
:1000F800010E041604500112000E02121950020DCE
:10010800250EF324D96E000EF420DA6E01C0DEFF4E
:1001180002C0DDFFF80E016EFF0E026E19061928E7
:10012800036E046A0150032602500422035004108F
:10013800D8A4C5D780A002D0838801D08398000EA8
:10014800176E25502610D8B406D0FF0E2614D8A452
:1001580002D0010E176E17B002D0839401D08384A9
:100168009E92838616C048F015C047F014C046F02A
:1001780013C045F012C0F5FF11C0F8FF10C0F7FF1B
:100188000FC0F6FF0EC0F4FF0DC0F3FF0CC0DAFF7E
:100198000BC0D9FF0AC0E2FF09C0E1FF08C0EAFFAF
:1001A80007C0E9FF06C0FBFF05C0FAFF4592110032
:1001B800AAEF01F01F502010D8B41200030E1F241C
:1001C8000001606F000E2020616F60516111D8B48A
:1001D80012001FC01AF020C01BF0080E1C6EECECB9
:1001E80001F01FC01AF020C01BF021C01CF022C073
:1001F8001DF0D9EC01F020EE03F01F50D926205055
:10020800DA2223C0DFFF20EE04F01F50D926205049
:10021800DA2224C0DFFF20EE01F01F50D92620503B
:10022800DA22020EDE6E000EDD6E12001B501C106C
:10023800D8B4120020EE01F01B50D9261C50DA2247
:10024800DECF1FF0DDCF20F0030E1B24216E000E41
:100258001C20226E1BC0D9FF1CC0DAFFDF380F0B31
:100268001D6E1BC0D9FF1CC0DAFFDF500F0B1E6EBE
:100278001E38F00B1D100CEC02F009D021C0D9FF7C
:1002880022C0DAFFDF500CEC02F0214A222A1F06B6
:10029800D8A020061F28F2E12028D8B41200EED7F3
:1002A800F29E9B8C9B809B829B849B869B889B9ABF
:1002B800D388D38AD38CFC0ED316000E0F01386F67
:1002C800000E396F000E3A6F000E3B6F926893680C
:1002D800959295949596959883828394838683982E
:1002E800800EBB6EBA50870B1809BA6E030EBA128D
:1002F800BA849D829E92F28CFEEC01F0F28E12007E
:1003080054EC01F0250E1A6E000E1B6E000E1D6EC9
:10031800000E1C6E000E1F6E1E0E1E6EC3EC01F04A
:10032800620E1F6E000E206E000E226E000E216EF1
:100338003C0E236E7F0E246EDEEC00F08392620E7C
:100348001B6E000E1C6E1AEC01F0F9D7240EF66E27
:10035800040EF76E000EF86E0900F5CF43F00900A1
:10036800F5CF44F000EE25F01E0EEE6AE806FDE13A
:1003780045904592000EF86E000184EF01F01AC016
:1003880020F01BC021F008D020C0D9FF21C0DAFF1F
:100398001CC0DFFF204A212A1E06D8A01F061E28DF
:1003A800F3E11F28D8B41200EFD71A501B10D8B4A5
:1003B80012001CC01EF00F0E1E161AC0D9FF1BC05B
:1003C800DAFF1E3ADF501E180F0B1E18DF6E1200E0
:1003D8001A501B10D8B412001CC01DF00F0E1D16A9
:1003E8001AC0D9FF1BC0DAFFDF501D18F00B1D180B
:1003F800DF6E1200AC98AC9CAB8E1F0EAF6E000E79
:10040800B06EAC94B896948E948CAB88AC8A12007B
:0E0418001A6E9EA8FED71AC0ADFF12003C005F
:020000040020DA
:08000000FFFFFFFFFFFFFFFF00
:020000040030CA
:0E000000FF391F3FFFBF85FF0FC00FE00F400D
:00000001FF
